:1000000012C0189518951895189518951895189563
:100010005CC5CEC118951895189518951895189522
:100020001895189518958FE58DBFC8E3E0E24E2E20
:1000300084E08EBFD4E0F4E05F2EA89584B7082E4C
:10004000877F84BF88E1992781BD91BDEEEFF3E002
:10005000A0E6B0E088278D933197E9F76624A09851
:10006000A89AA198A99AA298AA9A8FEF81BB8FEF1C
:1000700087BB86E886B980E487B981E08093620017
:1000800000916200063010F009F015C08BE090E09E
:10009000A2E6B0E0AD90BB24A3E6B0E0AA0CBB1C86
:1000A000AA0DBB1D8D939C93A2E6B0E08C918F5F4F
:1000B0008C9308F4E5CFEAE1F0E0A2E9B0E091E04A
:1000C0001ED9989957C081E0809362000091620028
:1000D000083C10F009F04EC000916200063909F0AA
:1000E0003CC080918C00806880938C00A2E9B0E0D5
:1000F0008C9198E089278C93EAE1F0E0A2E9B0E0E6
:1001000091E07BE7EBD800919200003009F00EC03F
:1001100092989698C798C2989098C6989798C598BC
:10012000939A949A919A959AC09AC19A0091920042
:10013000083009F00EC0929A969AC79AC29A909A7D
:10014000C69A979AC59A9398949891989598C098BA
:10015000C1988CED95E0AED70DC0989B01C00AC048
:100160008AE090E0A7D7A2E6B0E08C918F5F8C93F5
:1001700008F4ACCFE4E1F0E0A0E1B0E0BDD80F3F7F
:1001800009F040C086E990E0A5E7B0E08D939C932C
:1001900084E690E0ABE7B0E08D939C9380E08093A1
:1001A00092008BEB80938F0087E780939000E5E0CF
:1001B000F0E0A5E7B0E092E07BE790D8EEE0F0E079
:1001C000ABE7B0E092E07BE789D8E0E1F0E0AFE8B0
:1001D000B0E091E07BE782D8E1E1F0E0A0E9B0E0B7
:1001E00091E07BE77BD8EAE1F0E0A2E9B0E091E0C2
:1001F0007BE774D8E4E1F0E0A0E1BB2784E68C93D0
:100200007BE769D8E5E0F0E0A5E7B0E092E077D8D9
:10021000EEE0F0E0ABE7B0E092E071D8E0E1F0E0D2
:10022000AFE8B0E091E06BD8E1E1F0E0A0E9B0E048
:1002300091E065D882E083BF80E08FBD81E08EBD14
:10024000789489B7816089BF89B7846089BF82E06B
:1002500083BF81E08EBD379A81E080937D0081E08D
:1002600080937E00009162000A3010F009F001C016
:100270006AC0882783BF8EB5887F8EBD07B1007F97
:10028000056007B926D7A1E7B0E08D939C93A1E75D
:10029000B0E00D911C9142E050E0C9D6A1E7B0E07A
:1002A0004D935C93A1E7B0E00D911C91043F51E0A8
:1002B000150714F009F001C006C084EF91E0A1E732
:1002C000B0E08D939C9307B1007F046007B901D71C
:1002D000A7E7B0E08D939C93E7E7F0E0D190E08052
:1002E0008FEFE7FE8827F82E082F59D7A9E9B0E04D
:1002F00087D7ECE0F3E1CBD7E9E9F0E031D792D74B
:10030000EDE0F0E0A9E9B0E0DAD7E9E9F0E0F4D611
:10031000A7E7B0E0EE0C000FE794DD92EC92A7E7C0
:10032000B0E00D911C91073E53E0150714F009F061
:1003300001C006C087EE93E0A7E7B0E08D939C93E1
:1003400080E08093620082E083BF81E08EBDA5E7FC
:10035000B0E04D915C91A1E7B0E00D911C910417C4
:1003600015070CF001C003C080E080937D00009170
:100370007D00013009F002C0C39A01C0C398ABE709
:10038000B0E04D915C91A7E7B0E00D911C9104178E
:1003900015070CF001C003C080E080937E0000913F
:1003A0007E00013009F002C0C49A01C0C4985ACF3F
:1003B0000F921F922F923F924F925F927F92AF9235
:1003C000BF920F931F932F933F934F935F936F931E
:1003D0007F938F939F93AF93BF93CF93DF93EF93CD
:1003E000FF938FB78F9300918B00003081E009F469
:1003F00080E08F93ACE8B0E08C9185FB81E00EF457
:1004000080E09F918923882309F403C0ADE8B0E020
:10041000FDD5ADE8B0E00D911C9108355BE1150705
:1004200010F009F001C015C080E090E0ADE8B0E048
:100430008D939C9380E080938B00E5E0F0E0A5E74E
:10044000B0E092E05CD7EEE0F0E0ABE7B0E092E045
:1004500056D7882783BF00918B00003009F011C068
:10046000A1E7B0E08D919C91A5E8B0E08D939C93BD
:10047000A7E7B0E08D919C91A7E8B0E08D939C93A5
:1004800027C0023009F011C0A5E7B0E08D919C9122
:10049000A5E8B0E08D939C93A7E7B0E08D919C9187
:1004A000A7E8B0E08D939C9313C0043009F010C00E
:1004B000A1E7B0E08D919C91A5E8B0E08D939C936D
:1004C000ABE7B0E08D919C91A7E8B0E08D939C9351
:1004D000ACE8B0E08C9183FB0EF44FC0A5E8B0E02F
:1004E0008D919C91AFE7B0E08D939C93AFE7B0E026
:1004F0008D919C91A3E8B0E08D939C9383E08093D1
:1005000063004091630001E0041710F009F025C07A
:10051000AFE7B0E00D911C914AE050E088D5A3E62A
:10052000B0E0AD90BB24A3E6B0E0AA0CBB1CAA0DC2
:10053000BB1D0D931C93AFE7B0E00D911C914AE0F9
:1005400050E075D5AFE7B0E04D935C9380916300C8
:1005500081508093630008F0D4CFA3E8B0E00D9100
:100560001C91043650E015070CF401C006C08BE066
:1005700090E0A5E6B0E08D939C93ACE8B0E08C9160
:1005800082FB0EF43FC0A7E8B0E08D919C91A1E8FA
:10059000B0E08D939C93A1E8B0E08D919C91A3E88D
:1005A000B0E08D939C9386E080936300409163005C
:1005B00004E0041710F009F025C0A1E8B0E00D91A7
:1005C0001C914AE050E033D5A3E6B0E0AD90BB24E7
:1005D000A3E6B0E0AA0CBB1CAA0DBB1D0D931C9397
:1005E000A1E8B0E00D911C914AE050E020D5A1E8CF
:1005F000B0E04D935C9380916300815080936300E1
:1006000008F0D4CF00919200003009F007C0939811
:10061000949891989598C098C19806C0939A949A86
:10062000919A959AC09AC19AA0E6B0E08C918F5F9A
:100630008C9300916000063010F009F001C003C0F7
:1006400081E08093600080E08093610090D1A4E617
:10065000B0E08C9180FBA2E3B0E08C9182F98C93A6
:1006600086D1A4E6B0E08C9180FBA2E3B0E08C914F
:1006700086F98C937CD1A4E6B0E08C9180FBA8E352
:10068000B0E08C9187F98C9372D1A4E6B0E08C91A4
:1006900080FBA8E3B0E08C9182F98C9368D1A4E64A
:1006A000B0E08C9180FBA2E3B0E08C9180F98C9358
:1006B0005ED1A4E6B0E08C9180FBA8E3B0E08C9121
:1006C00086F98C9354D1A4E6B0E08C9180FBA2E330
:1006D000B0E08C9187F98C9300916000013009F0B3
:1006E0002FC000919200003009F013C0919AACE83D
:1006F000B0E08C9183FB0EF40AC0AFE8B0E08C91BF
:1007000083FBA8E3B0E08C9185F98C9301C0C59A76
:1007100016C09198ACE8B0E08C9183FB0EF40EC04B
:10072000AFE8B0E08C9183FBA8E3B0E08C9185F951
:100730008C9388B390E2892788BB01C0C598F9C023
:10074000023009F02FC000919200003009F013C070
:10075000949AACE8B0E08C9183FB0EF40AC0AFE849
:10076000B0E08C9182FBA8E3B0E08C9185F98C938A
:1007700001C0C59A16C09498ACE8B0E08C9183FB98
:100780000EF40EC0AFE8B0E08C9182FBA8E3B0E0BD
:100790008C9185F98C9388B390E2892788BB01C03E
:1007A000C598C7C0033009F02FC0009192000030F7
:1007B00009F013C0939AACE8B0E08C9183FB0EF47F
:1007C0000AC0AFE8B0E08C9181FBA8E3B0E08C9167
:1007D00085F98C9301C0C59A16C09398ACE8B0E037
:1007E0008C9183FB0EF40EC0AFE8B0E08C9181FBDE
:1007F000A8E3B0E08C9185F98C9388B390E28927C7
:1008000088BB01C0C59895C0043009F02FC0009185
:100810009200003009F013C0C19AACE8B0E08C91AE
:1008200082FB0EF40AC0A0E9B0E08C9183FBA8E340
:10083000B0E08C9185F98C9301C0C59A16C0C1981F
:10084000ACE8B0E08C9183FB0EF40EC0A0E9B0E000
:100850008C9183FBA8E3B0E08C9185F98C9388B3ED
:1008600090E2892788BB01C0C59863C0053009F0B4
:100870002FC000919200003009F013C0C09AACE87C
:10088000B0E08C9182FB0EF40AC0A0E9B0E08C913C
:1008900082FBA8E3B0E08C9185F98C9301C0C59AE6
:1008A00016C0C098ACE8B0E08C9183FB0EF40EC08B
:1008B000A0E9B0E08C9182FBA8E3B0E08C9185F9CF
:1008C0008C9388B390E2892788BB01C0C59831C05A
:1008D000063009F02EC000919200003009F013C0DC
:1008E000959AACE8B0E08C9182FB0EF40AC0A0E9C6
:1008F000B0E08C9181FBA8E3B0E08C9185F98C93FA
:1009000001C0C59A16C09598ACE8B0E08C9183FB05
:100910000EF40EC0A0E9B0E08C9181FBA8E3B0E03A
:100920008C9185F98C9388B390E2892788BB01C0AC
:10093000C59882E083BF8F918FBFFF91EF91DF91C8
:10094000CF91BF91AF919F918F917F916F915F9167
:100950004F913F912F911F910F91BF90AF907F903A
:100960005F904F903F902F901F900F901895A0E6AA
:10097000B0E0AD90BB24A3E6B0E0AA0CBB1CAA0D6E
:10098000BB1D0C9147E0049FA4E6B0E00C920091DF
:10099000610040916400040FA4E6B0E00C93009164
:1009A0009200003009F00AC0EAEDF9E0A4E6B0E0F8
:1009B0008C919927A4E6B0E07FD409C0E2E5FAE083
:1009C000A4E6B0E08C919927A4E6B0E075D4A1E646
:1009D000B0E08C918F5F8C930895000000000000C0
:1009E00001010000010101010000010000010000FF
:1009F00000000001010001000001010000000100F1
:100A000000010000000100000000000000000101E2
:100A100001010000000000000000000000010000D3
:100A200001010101010100010101010101010101B7
:100A300001000000010101000100010000010101AD
:100A4000000000000101000000000101010100019F
:100A5000000001010101010100000101000000008E
:100A6000010100010100010101010100000100017B
:100A7000010000010101000101000101010001016B
:100A8000010101010101000000000101010101015A
:100A9000010101010100010100000000000001004E
:100AA0000000000000000000000101010000000142
:100AB000000100010100000001010101000001012D
:100AC000010100000000010001000F921F922F920F
:100AD0003F924F925F927F92AF92BF920F931F937C
:100AE0002F933F934F935F936F937F938F939F9336
:100AF000AF93BF93CF93DF93EF93FF938FB78F9312
:100B0000A2E6B0E08C918F5F8C938EB5887F8EBD0E
:100B100000917D00003081E009F080E08F9300912A
:100B20007E00003081E009F080E09F91892B8823CE
:100B300009F41AC0A3E3B0E00C9101FB81E00EF4CC
:100B400080E08F93A3E3B0E00C9102FB81E00EF410
:100B500080E09F91892B882309F406C081E080936F
:100B60007D0081E080937E00A3E3B0E00C9100FB68
:100B700081E00EF480E08F93ACE8B0E08C9187FBCD
:100B800081E00EF480E09F9189238F93A3E3B0E08E
:100B90000C9101FB81E00EF080E09F9189238F93FF
:100BA000A3E3B0E00C9102FB81E00EF080E09F91A6
:100BB0008923882309F401C0B7D0ACE8B0E08C9158
:100BC00084FB81E00EF080E08F93A3E3B0E00C9112
:100BD00000FB81E00EF080E09F918923882309F4D7
:100BE00006C0999901C064D19A9901C0A0D1A3E32C
:100BF000B0E00C9100FB81E00EF480E08F93A3E362
:100C0000B0E00C9101FB81E00EF480E09F9189231C
:100C10008F9300918B00003081E009F080E09F917C
:100C200089238F93ACE8B0E08C9186FB81E00EF4D1
:100C300080E09F918923882309F401C0BBD1A3E3FD
:100C4000B0E00C9100FB81E00EF480E08F93A3E311
:100C5000B0E00C9102FB81E00EF480E09F918923CB
:100C60008F9300918B00003081E009F080E09F912C
:100C700089238F93ACE8B0E08C9186FB81E00EF481
:100C800080E09F918923882309F401C0A9D1A3E3BF
:100C9000B0E00C9100FB81E00EF080E08F93A3E3C5
:100CA000B0E00C9101FB81E00EF080E09F91892380
:100CB0008F93A3E3B0E00C9102FB81E00EF080E0A3
:100CC0009F918923882309F408C080918C008F7735
:100CD00080938C0084E680939800989B05C0809157
:100CE0008C008F7B80938C0081E08EBD82E083BF7F
:100CF0008F918FBFFF91EF91DF91CF91BF91AF9116
:100D00009F918F917F916F915F914F913F912F9123
:100D10001F910F91BF90AF907F905F904F903F9049
:100D20002F901F900F901895789489B7816089BF94
:100D300082E083BF80918C00806180938C008091E1
:100D40008C00806880938C0080E090E0ADE8B0E09B
:100D50008D939C93ABE8B0E08C918E5F8C93009167
:100D60008B00043010F009F001C003C080E08093D4
:100D70008B0000918B00003009F043C080918C0003
:100D8000886080938C0080918C00846080938C00BC
:100D90008AE090E0A5E6B0E08D939C938AE090E035
:100DA000A7E6B0E08D939C938AE090E0A9E6B0E0DE
:100DB0008D939C938AE090E0ABE6B0E08D939C939A
:100DC0008AE090E0ADE6B0E08D939C938AE090E0FD
:100DD000AFE6B0E08D939C9380918C008F7E8093E2
:100DE0008C0084EF91E066D18EB5887F8EBD882718
:100DF00083BFEEE0F0E0ABE7B0E092E07BE76ED2DD
:100E00004CC0023009F020C080918C008860809333
:100E10008C0081E090E0A9E6B0E08D939C938EE099
:100E200090E0A7E6B0E08D939C9380E090E0A5E68B
:100E3000B0E08D939C9384EF91E03CD18EB5887F98
:100E40008EBD882783BF29C0043009F026C0809159
:100E50008C00846080938C0082E090E0AFE6B0E08C
:100E60008D939C938EE090E0ADE6B0E08D939C93E3
:100E700080E090E0ABE6B0E08D939C9384EF91E04E
:100E800019D18EB5887F8EBD882783BFE5E0F0E05D
:100E9000A5E7B0E092E07BE721D280918C00877FCC
:100EA00080938C0080918C008B7F80938C000895C0
:100EB000789489B7816089BF82E083BF80E090E049
:100EC000ADE8B0E08D939C93009198000A3010F04B
:100ED00009F001C005C0A8E9B0E08C9185508C9361
:100EE00000918B00023009F00DC0A5E7B0E00D9134
:100EF0001C91043F51E0150708F003C0A5E7B0E0DE
:100F000085D00FC0043009F00CC0ABE7B0E00D9104
:100F10001C91073E53E0150708F003C0ABE7B0E0B3
:100F200075D0A8E9B0E08C919927C4D00895789441
:100F300089B7816089BF82E083BF80E090E0ADE83F
:100F4000B0E08D939C93009198000A3010F009F066
:100F500001C005C0A8E9B0E08C9185508C93009148
:100F60008B00023009F00FC0A5E7B0E00D911C9195
:100F7000003050E0150710F009F001C003C0A5E7EC
:100F8000B0E04BD011C0043009F00EC0ABE7B0E0C8
:100F90000D911C91003050E0150710F009F001C0D0
:100FA00003C0ABE7B0E039D0A8E9B0E08C91992755
:100FB00081D0089580918C00806480938C0091E0B2
:100FC000AFE8B0E08FD08EB5887F8EBD882783BF15
:100FD000E0E1F0E0AFE8B0E091E07BE77FD1089599
:100FE00080918C00806480938C0091E0A0E9B0E057
:100FF00079D08EB5887F8EBD882783BFE1E1F0E090
:10100000A0E9B0E091E07BE769D10895ED91FC9112
:10101000EF5FFF4FFC93EE930895ED91FC91E1504B
:10102000F040FC93EE93089500FC10D0089503D097
:101030001ED001F8F9CF0024E89457FF02C009D070
:10104000689400F80BD010F80124089502D009D05C
:101050000895509540954F5F5F4F0895E89417FFAE
:101060000895009510950F5F1F4F68940895352FD0
:10107000242FE894452B11F468940895512F402FA4
:101080000027112780E1440F551F001F111F021B6D
:10109000130B416018F4020F131F4E7F8A9599F7C6
:1010A00008953197F1F70895689462F80895E894E7
:1010B00062F80895EF93FF93EE27E82BE92B31F0C8
:1010C000E0EDF7E03197F1F70197D1F7FF91EF915C
:1010D0000895369A3699FECF369A3699FECF84B166
:1010E00095B10895903039F08C91880F08F48160A3
:1010F0009A95D9F78C93089533D0992711278F2D7E
:10110000880F80E8F82A802F881F08F41FEF41F02D
:101110008F57082F07FD04C0003240F08FEF01C049
:101120008827982FD82EE82EF82E09C08FE1801B33
:10113000082FF694E794D79497950A95D1F7112341
:1011400051F09095D094E094F09481E0980F882726
:10115000D81EE81EF81E0F2DFE2CED2CD92E08955A
:10116000D190E190F19001910895102F90E8FF0C3B
:10117000001F0927990FF7941078652F90E8440F06
:10118000551F5927990F4795607800380895FF0C2F
:1011900090E89027110F9795F794092F0895102F35
:1011A000BD2CDE2CEF2CF02E11234AF4B094D094F9
:1011B000E094F0949FEFB91AD90AE90AF90A0EE10E
:1011C000FF2039F4FE2CED2CDB2CBB240850C2F799
:1011D00023C032F00A95BB0CDD1CEE1CFF1CF9CFBE
:1011E00001D0D5CFB7FE089590E8B91611F4D0FE1E
:1011F00008959FEFD91AE90AF90A09F403950895A9
:10120000DD92ED92FD920C9308959FE7092FF92A44
:101210009FEFD92EE92E0895DD24EE24FF24002728
:1012200011270895A2DFC1F35038B1F316270058F3
:1012300050580894051F12F418F4E7CF08F0ECCFCB
:101240000BD0FF202AF0BB0CDD1CEE1CFF1C9FCF37
:101250000F5F0BF4DACF9BCF9F929924AA24BB2473
:10126000992788E1990CAA1CBB1CDD1CEE1CFF1CF5
:1012700030F4920EA31EB41ED91EE91EF91E8A95E3
:1012800089F79F900895C895319600200895FBDF57
:10129000202DF9DF302DF7DF402DF5DF502D08959B
:1012A00091E005C092E003C094E001C098E0EBDF5C
:1012B0000D929A95E1F70895E80FF91FF1CF94E0A8
:1012C00081918D939A95E1F70895E199FECFEEBB58
:1012D000FFBB3196089591E001C092E07B3751F455
:1012E0007FB7F894F2DF8D918DBBE29AE19A9A95DF
:1012F000C9F77FBF7727089591E001C092E0E5DF4D
:10130000E09A8DB38D939A95D1F708958F539C3FB2
:00000001FF
